:1064FA000A2A2A2A2A2A2A2A2A2A2A2A2A2A2A2A12
:10650A002A2A20CFE0F0E0ECE5F2F0FB20E0E4E01C
:10651A00EFF2E5F0E0202A2A2A2A2A2A2A2A2A2A17
:10652A002A2A2A2A2A2A2A2A0A00312E204D4143B7
:10653A0020E0E4F0E5F13A202025303262783A256D
:10654A00303262783A25303262783A2530326278CF
:10655A003A25303262783A25303262780A00322E91
:10656A0020495020E0E4F0E5F13A20202025627528
:10657A002E2562752E2562752E2562750A00332E28
:10658A0020D8EBFEE73A2020202020202025627523
:10659A002E2562752E2562752E2562750A00342E07
:1065AA0020CCE0F1EAE020F1E5F2E83A2025627534
:1065BA002E2562752E2562752E2562750A00352EE6
:1065CA0020495020E0E4F0E5F120F1E5F0E2E5F0C1
:1065DA00E0313A202562752E2562752E2562752EC8
:1065EA002562750A00362E20495020E0E4F0E5F1D4
:1065FA0020F1E5F0E2E5F0E0323A202562752E2539
:10660A0062752E2562752E2562750A00372E20D2F4
:10661A00E0E9EC2DE0F3F220EEF2E2E5F2E020F11F
:10662A00E5F0E2E5F0E03A2025627520282A3130CB
:10663A006D63290A00302E20CAEBFEF720E4EEF142
:10664A00F2F3EFE03A2025730A000AC7C0CFC8D197
:10665A00DC20466C6173680A000AC7E0EFE8F1FCC7
:10666A0020E7E0E2E5F0F8E5EDE0210A000820087D
:10667A00000A53696E636F6D4950205665722E2069
:10668A00322E3120434320282770272DE2F5EEE4ED
:10669A0020E220EAEEEDF4E8E3F3F0E0F2EEF0298E
:1066AA00000A3E20CAEEEDF4E8E3F3F0E0F6E8EE85
:1066BA00EDEDFBE920F0E5E6E8EC0A0A00203C49AA
:1066CA003E20203A20CFEEEAE0E7E0F2FC20EFE0BD
:1066DA00F0E0ECE5F2F0FB0A00203C536E3E203A73
:1066EA0020C7E0E4E0F2FC20EFE0F0E0ECE5F2F0B5
:1066FA0020276E270A00203C4B3E20203A20C7E084
:10670A00E3F0F3E7E8F2FC20EDEEE2F3FE20EAEE36
:10671A00EDF42E20E8E720F4E0E9EBE00A00203C63
:10672A00443E20203A20D0E0F1EFE5F7E0F2E0F233
:10673A00FC20EDEEE2F3FE20EAEEEDF42E0A002054
:10674A003C573E20203A20C7E0EFE8F1E0F2FC2077
:10675A00E8E7ECE5EDE5EDE8FF0A00203C4C3E20D9
:10676A00203A20C7E0E3F0F3E7E8F2FC20EFF0EE8E
:10677A00E3F0E0ECECF32028586D6F64656D290AAC
:10678A0000203C453E20203A20C2FBF5EEE40A00F8
:10679A003E20C2E2E5E4E8F2E520EAEEECE0EDE4D0
:1067AA00F33A20000AC2E2E5E4E8F2E520274D4187
:1067BA004320E0E4F0E5F15B2562645D273A202599
:1067CA0030326278202D3E0078000AC2E2E5E4E821
:1067DA00F2E52027495020E0E4E0EFF2E5F0E05B43
:1067EA002562645D273A20256275202D3E007500DA
:1067FA000AC2E2E5E4E8F2E52027D8EBFEE75B25EA
:10680A0062645D273A20256275202D3E000AC2E2A5
:10681A00E5E4E8F2E52027CCE0F1EAF3D1E5F2E895
:10682A005B2562645D273A20256275202D3E000AA9
:10683A00C2E2E5E4E8F2E52027495020F1E5F0E27A
:10684A00E5F0E0315B2562645D273A202562752018
:10685A002D3E000AC2E2E5E4E8F2E520274950208D
:10686A00F1E5F0E2E5F0E0325B2562645D273A206B
:10687A00256275202D3E000AC2E2E5E4E8F2E52031
:10688A0027C2F0E5ECFF20EEE6E8E4E0EDE8FF20C1
:10689A00EEF2E2E5F2E0273A20256275202D3E006D
:1068AA000AC2E2E5E4E8F2E520EAEBFEF720E4EECC
:1068BA00F1F2F3EFE028E4EE203720F1E8ECE229E8
:1068CA003A0A2D3E000A204572726F72210A000AA6
:1068DA00C8C4C5D220C7C0CFC8D1DC2120C6C4C80D
:1068EA00D2C521000AC7C0CFC8D1DC20C7C0C2C5E3
:1068FA00D0D8C5CDC0210A000A20000ACA20EFF06C
:10690A00E8E5ECF320E3EEF2EEE2210A000A454F55
:10691A0054210A000AD4E0E9EB20E7E0E3F0F3E6C9
:10692A00E5ED210A00CEF8E8E1EAE0210A000AD4FE
:10693A00E0E9EB20EFEEEBF3F7E5ED2120C7E0EF1E
:10694A00E8F1FC20E220454550524F4D210A003C17
:10695A004D41433D003C4130313D003C4130323DE8
:10696A00003C4130333D003C4130343D003C413035
:10697A00353D003C4130363D000ACAEEEDF4E8E30D
:10698A00F3F0E0F6E8FF20E7E0EFE8F1E0EDE021E0
:02699A000A00F1
:1077DB00E4FF7E0374142EF582E43460F583E02F0E
:1077EB00FF0EBE83EF74142EF582E43460F583E054
:0577FB00FEC3EF9EFF3C
:017800002265
:10773D00C2ADE4F5C9D2CDD2CCC2C9C2CAF5CDF520
:10774D00CC75CBFF75CAB885CBCD85CACCD29ED2B0
:10775D009CD2CAE59924FF92CAC2ACC298C2993094
:06776D0099032098FA22A6
:0778BF003098FDAF99C2985B
:0178C600229F
:0678A5001278BFEFF5228E
:0878AB008F993099FDC299226A
:10789500AE07BE0A057F0D1278ABAF061278AB2294
:10740E007BFF7A6479FA1269FE7BFF7A6579349094
:10741E0061A2E0F536A3E0F537A3E0F538A3E0F579
:10742E0039A3E0F53AA3E0F53B1269FE7BFF7A65DE
:10743E0079689061A8E0F536A3E0F537A3E0F5385A
:10744E00A3E0F5391269FE7BFF7A65798890619A1F
:10745E00E0F536A3E0F537A3E0F538A3E0F53912F1
:10746E0069FE7BFF7A6579A890619EE0F536A3E010
:10747E00F537A3E0F538A3E0F5391269FE7BFF7A04
:10748E006579C89061B1E0F536A3E0F537A3E0F574
:10749E0038A3E0F5391269FE7BFF7A6579EF9061CA
:1074AE00B5E0F536A3E0F537A3E0F538A3E0F539FE
:1074BE001269FE7BFF7A6679169061B9E0F5361295
:1074CE0069FE7536017537617538CB7BFF7A667943
:0474DE003F0269FE02
:0675AF008E298F2A8D2BAE
:1075B500E4F530F531F52EF52FE52B60097BFF7AE3
:1075C5006679541269FEE4F52CF52DE529C4F854C5
:1075D500F0C868FEE52AC4540F48FFC3E52D9FE5B2
:1075E5002C9E5040AE30AF31AD07AC067B10AF2FAF
:1075F500AE2E1277A774102531F531E43530F5300C
:107605007410252FF52FE4352EF52EE52B600BE5AF
:107615002D543F70057F231278AB052DE52D70ABFA
:10762500052C80A7E529C4F854F0C868FEE52AC4EE
:10763500540F48C4F8540FC868FFEEC454F048FE10
:10764500C3E52A9FFFE5299EAC30AD31AB07AF2FCF
:10765500AE2E1277A7E52B60097BFF7A6679631258
:0276650069FEBC
:017667002200
:0474E2007E677FF84A
:0474E6008E298F2A32
:1074EA00E4F52B7400252BF582E43460F583E4F08F
:1074FA00052BE52BB408ECE4F52B1278BFEFF52C3D
:10750A00640A6005E52CB40D0F7400252BF582E49E
:10751A003460F583E4F08044E52CB40824E52BD3E9
:10752A009400402F7BFF7A6679771269FE152B74D7
:10753A0000252BF582E43460F5837420F0152B8046
:10754A00127400252BF582E43460F583E52CF0FFF4
:10755A001278AB052BE52BC39408409EE52B7002ED
:10756A00FF22852A82852983E493B4781E906000DD
:10757A00E0FF127773EFC454F0FEC006906001E09A
:10758A00FF127773D0E02FF5088017753100753236
:10759A0000753300E4F5347B017A607900127136A4
:0475AA008F087F01C6
:0175AE0022BA
:10600300752501C2AF907FFEE0B4FF047F018002DB
:106013007F00907FFDE0B4AA047E0180027E00EE43
:106023005FFF907FFFE0B455047E0180027E00EEA7
:106033005F6028E4907FFDF0A3F0A3F0907FF0E091
:10604300FEA3E0FF4E6005E4FD1275AF7BFF7A000F
:1060530079008B268A27892812700112773DC2980E
:106063007BFF7A66797B1269FE30980F7BFF7A009B
:1060730079008B268A278928127001E4F523E4F539
:10608300242098030264C51278BFEFF522645060A0
:1060930009E522647060030264B6AF221278AB7F15
:1060A3000A1278ABE4F523E5232401FFE433FE125F
:1060B3007820749A2523F582E43461F583EFF005A3
:1060C30023E523C3943F40DFE4F523E523247FFF47
:1060D300E433FE12782074142523F582E43461F549
:1060E30083EFF00523E523C3948040DFE4906193BD
:1060F300F0E52570030264C57BFF7A6679AB12690C
:10610300FE7BFF7A6679C71269FE7BFF7A6679E3C5
:106113001269FE7BFF7A6779001269FE7BFF7A675B
:1061230079281269FE7BFF7A6779491269FE7BFF42
:106133007A6779651269FE7BFF7A67798B1269FE4C
:106143007BFF7A67799A1269FE1278A5E522126FAE
:10615300DB646F4464004561824964694B64634C4A
:10616300618853640657646F64640065618269647F
:10617300696B64636C618873640677000060F41272
:10618300740E0260F41278A5E522126FDB634B30C4
:1061930061AC3161EF32622E33626D3462AC3562D1
:1061A300EB36632A37000063F8E4F522E522C39453
:1061B3000640030260F47BFF7A6779AE852236746A
:1061C300A22522F582E43461F583E0F5371269FEF6
:1061D3007E677FD21274E6EF600E74A22522F582E9
:1061E300E43461F583E508F0052280C0E4F522E597
:1061F30022C3940440030260F47BFF7A6779D48559
:10620300223674A82522F582E43461F583E0F5375C
:106213001269FE1274E2EF600E74A82522F582E47F
:106223003461F583E508F0052280C4E4F522E52214
:10623300C3940440030260F47BFF7A6779FA8522F2
:1062430036749A2522F582E43461F583E0F537123A
:1062530069FE1274E2EF600E749A2522F582E4342B
:1062630061F583E508F0052280C4E4F522E522C345
:10627300940440030260F47BFF7A68791785223621
:10628300749E2522F582E43461F583E0F5371269C3
:10629300FE1274E2EF600E749E2522F582E43461EF
:1062A300F583E508F0052280C4E4F522E522C394D2
:1062B3000440030260F47BFF7A68793985223674DF
:1062C300B12522F582E43461F583E0F5371269FEE6
:1062D3001274E2EF600E74B12522F582E43461F5A5
:1062E30083E508F0052280C4E4F522E522C3940483
:1062F30040030260F47BFF7A68795D85223674B5CA
:106303002522F582E43461F583E0F5371269FE1244
:1063130074E2EF600E74B52522F582E43461F583EF
:10632300E508F0052280C47BFF7A6879819061B922
:10633300E0F5361269FE1274E2EF70030260F49026
:1063430061B9E508F00260F47BFF7A6879AA126903
:10635300FEE4F52374CB2523F582E43461F583E46D
:10636300F00523E523B408ECE4F5231278BFEFF539
:1063730022640A6005E522B40D0F74CB2523F58250
:10638300E43461F583E4F08044E522B40824E52392
:10639300D39400402F7BFF7A6679771269FE152329
:1063A30074CB2523F582E43461F5837420F015233F
:1063B300801274CB2523F582E43461F583E522F062
:1063C300FF1278AB0523E523C39408409E9061CB6D
:1063D300E0642060030260F4F523E523C3940840DE
:1063E300030260F474CB2523F582E43461F583E47E
:1063F300F0052380E57BFF7A6879CF805DE4F5259E
:106403000260F47BFF7A6879D91269FEE4F523E52B
:10641300232401FFE433FE749A2523F582E43461D7
:10642300F583E0FD12783C0523E523C3943F40DF69
:10643300E4F523E523247FFFE433FE74142523F5D9
:1064430082E43461F583E0FD12783C0523E523C340
:10645300948040DF7BFF7A6879EE1269FE0260F474
:106463001278C70260F4126CF80260F47BFF7A6959
:1064730079021269FE906194E4F0A374FFF0E4F5ED
:1064830023C3E52394D07480948740030260F4E52A
:1064930022F470030260F4E52270030260F41278C0
:1064A3006D8F221278ABE522642170030260F4053C
:1064B3002380CE7BFF7A0079008B268A27892812D6
:1064C30070017F057E001278010524E524C3941929
:1064D30050030260847F2E1278AB0523E523C39417
:1064E3000A50030260817BFF7A0079008B268A279A
:0764F300892812700180FEF0
:10780100E4FDFCC3ED9FEC9E5014E4FBFA0BBB00BE
:0E781100010AEBF44A70F60DBD00010C80E593
:01781F002246
:1072DA00753160753217E4F52FF530C2017BFF7AFC
:1072EA006979051269FE2098247F151278ABE4F5B6
:1072FA002BF52CC3E52C9420E52B648094CE50E624
:10730A002098E3052CE52C70EA052B80E6D200755F
:10731A002E01E599B404097BFF7A6979170274068C
:10732A003001030273E3C3E53094C0E52F945D4056
:10733A00030273E3E4F52D20983AE4F52BF52CAE1D
:10734A002BAF2CEE3395E0FDFCE47B407A9CF9F8F8
:10735A00D3126F5F400D20980A052CE52C70E005CA
:10736A002B80DC20980E3000047F0680027F1512E5
:10737A0078AB80C3C298E52D7009E599B40404D2AC
:10738A000180177414252DF582E43460F583E5999C
:10739A00F0052DE52DC39484409D1277DBEF600A3A
:1073AA007F151278ABC20002732AD200906015E0F2
:1073BA00B52E1E052EAE31AF32AD07AC067B80AFBF
:1073CA0030AE2F1277A774802530F530E4352FF5CB
:1073DA002F7F061278AB02732A7F201278ABE4F56E
:1073EA002BF52C209810052CE52C7002052BB420C7
:1073FA00F2E52BB44EED7BFF7A69791E1269FE7EA7
:03740A00007F01FF
:01740D00225C
:0778C7001272DA8E298F2AEC
:0178CE002297
:10777300EFC39430400BEFD394395005EF24D0FF7F
:1077830022EFC39461400BEFD394665005EF24A915
:10779300FF22EFC39441400BEFD394465005EF24EF
:0477A300C9FF2222D6
:10786D00906194E475F001126F49906194E0FEA36C
:06787D00E0FF127820225A
:1078550012786D127773EFC454F0FEC00612786D7E
:08786500127773D0E02FFF221F
:1076E80012786D906000EFF012786D906001EFF005
:1076F80012786D906002EFF012786D906003EFF0F1
:1077080012786D906004EFF012786D906005EFF0DC
:1077180012786D906006EFF012786D906007EFF0C8
:10772800E4A3F0F531F532F533F5347B017A60796D
:05773800001271362271
:047668008E2E8F2FA4
:10766C00906194E4F0A374FFF012786DEF6069F40C
:10767C006066852F82852E83E493B507EC75300107
:10768C00E52F2530F582E4352EF583E493602590C3
:10769C006195E02530FF906194E03400FE12782073
:1076AC00E52F2530F582E4352EF583E493B50704F8
:1076BC00053080CCE52F2530F582E4352EF583E4BA
:1076CC009370A6E53024FFFFE434FF9061948FF0B3
:0B76DC00126F497E007F0122E4FEFFD8
:0176E7002280
:106CF8007BFF7A6979051269FE9061D9126FAA0043
:106D0800000000E4F529F52A209841D3E52A9400EB
:106D1800E529940040199061D9126F86EF2401FF8C
:106D2800E43EFEE43DFDE43CFC9061D9126F9E7F99
:106D3800E07E937D047C009061D9126F92D3126F2C
:106D48007540C57BFF7A69792F026F459061D9122A
:106D58006FAA000000001278BF8F2DE52D643C60FB
:106D680011052AE52A70020529C394C0E529945D16
:106D78004096900000E52DF0752900752A011278DB
:106D8800BF8F2D852A82852983E52DF06421601126
:106D9800052AE52A70020529C394D0E529940740FD
:106DA800DD7BFF7A6979381269FEE52A2401F52C22
:106DB800E43529F52BE4F529F52AC3E52A952CE5D0
:106DC80029952B501EE4252AFFE5293401FE852A42
:106DD80082852983E0FD12783C052AE52A70DB05C7
:106DE8002980D77E697F59127668EF4E6030127815
:106DF800559061A2EFF01278559061A3EFF01278E8
:106E0800559061A4EFF01278559061A5EFF01278D3
:106E1800559061A6EFF01278559061A7EFF07E6962
:106E28007F5F127668EF4E60201278559061A8EF68
:106E3800F01278559061A9EFF01278559061AAEF99
:106E4800F01278559061ABEFF07E697F6512766835
:106E5800EF4E60201278559061B1EFF0127855909E
:106E680061B2EFF01278559061B3EFF01278559057
:106E780061B4EFF07E697F6B127668EF4E60201286
:106E880078559061B5EFF01278559061B6EFF01231
:106E980078559061B7EFF01278559061B8EFF07EB1
:106EA800697F71127668EF4E602012785590619E66
:106EB800EFF012785590619FEFF01278559061A02D
:106EC800EFF01278559061A1EFF07E697F77127626
:106ED80068EF4E602012785590619AEFF01278555D
:106EE80090619BEFF012785590619CEFF012785505
:106EF80090619DEFF07E697F7D127668EF4E6008A5
:106F08001276E89061B9EFF0E4F529F52AE52A242C
:106F180001FFE43529FE749A252AF582E43461F5E7
:106F280083E0FD12783C052AE52A70020529C394FE
:106F380043E529940040D67BFF7A6979831269FE7C
:016F48002226
:0277A7008B3322
:1077A900A2AF9202C2AF85A23453A2FE8E838F820A
:1077B90005A28C838D827409127883E53353A2FE66
:1077C90043A22012788553A2DF8534A2A20292AF88
:0177D900FFB0
:0177DA00228C
:10782000E5D220E0FBC2AF438E2075D2028F828E5C
:0B78300083E0FFE4F5D2538EDFD2AFFF
:01783B00222A
:10783C00E5D220E0FBC2AF43D2028F828E83EDF003
:09784C0075D25063D250D2AF2274
:10788300F922C002C004C00612FFF0D006D004D013
:027893000222CF
:036000000278B370
:0C78B30078FFE4F6D8FD75814602600302
:106F4900C5F0F8A3E028F0C5F0F8E58215827002D3
:066F59001583E038F02270
:106F5F00EB9FF5F0EA9E42F0E99D42F0EC6480C8A9
:066F6F0064809845F02249
:106F7500EB9FF5F0EA9E42F0E99D42F0E89C45F072
:016F850022E9
:0C6F8600E0FCA3E0FDA3E0FEA3E0FF227E
:0C6F9200E0F8A3E0F9A3E0FAA3E0FB2282
:0C6F9E00ECF0A3EDF0A3EEF0A3EFF02266
:106FAA00A8828583F0D083D082126FC1126FC1127A
:106FBA006FC1126FC1E473E493A3C583C5F0C5839F
:106FCA00C8C582C8F0A3C583C5F0C583C8C582C831
:016FDA002294
:106FDB00D083D082F8E4937012740193700DA3A345
:106FEB0093F8740193F5828883E473740293686059
:066FFB00EFA3A3A380DF59
:067001008A838982E4731A
:10699C00E5422436F8E6054222783330090278368F
:1069AC00E475F0011270BC0270072002EB7F2ED24E
:1069BC00028018EF540F2490D43440D4FF30060BCF
:1069CC00EF24BFB41A0050032461FFE543600215A5
:1069DC00430546E5467002054530090D7833E475EC
:1069EC00F0011270BCEF02704D0278957403D2095D
:1069FC008003E4C209F5428B338A348935E4F543CC
:106A0C00F545F546E54360077F201269D780F5759B
:106A1C0044FFC203C202C204C205C207C208C20AB2
:106A2C001269A5FF700D3009057F001269E8AF46A9
:106A3C00AE4522B4255FC2D5C2061269A5FF24D08B
:106A4C00B40A00501A75F00A784330D50508B6FF21
:106A5C000106C6A426F620D5047002D20580D924DE
:106A6C00CFB41A00EF5004C2E5D206026BE8D20391
:106A7C0080C6D20280C0D20480BCD2D580BAD207E4
:106A8C0080B47F201269D72004077401B5430040FD
:106A9C00F112699CFF1269D7026A10D20AD20880DF
:106AAC009512699CFB12699CFA12699CF94A4B700D
:106ABC000679B97A6C7BFF20042EE543602A7E00B0
:106ACC008E8275830012702060060EEE654470F0A5
:106ADC00C2D5EBC0E0EAC0E0E9C0E0EE126C2FD00A
:106AEC00E0F9D0E0FAD0E0FB127007FF60AAEBC02F
:106AFC00E0EAC0E0E9C0E01269D7D0E02401F9D0A7
:106B0C00E03400FAD0E0FBE5440460DCD544D980E5
:106B1C00877BFF7A6C792BD204809C791080027968
:106B2C0008C208C20A8008D2D5790A8004790AC240
:106B3C00D5E544047002F544E4FAFDFEFF12699CAD
:106B4C00FC7B0820031312699CFD7B1030020A1297
:106B5C00699CFE12699CFF7B20EC3382D592D55048
:106B6C0013C3E43002069FFFE49EFEE42003039D62
:106B7C00FDE49CFCE4CBF8C203EC700CCFCECDCC86
:106B8C00E824F8F870F38017C3EF33FFEE33FEED13
:106B9C0033FDEC33FCEB33FB994002FB0FD8E9EBF4
:106BAC00300305F8D0E0C448B203C0E00AEC4D4E07
:106BBC004F78207B0070C2EAB5440040BCC0E012A4
:106BCC006C31D0F0D0E0200304C4C0E0C4B203C0E8
:106BDC00F01269C0D0F0D5F0EB026A10126FDB6ACC
:106BEC00AD536B27586A7E4C6A7A426B2B4F6B33D2
:0F6BFC00446B33496A93436B39556B1D466B1DD0
:106C0B00456B1D476CD9506A822D6A862E6AA92B5B
:106C1B006A8A236AA7206CC22A6A424800006AA1CA
:106C2B003F3F3F00790AA2D5200514300709B91060
:106C3B00020404B9080104A2D52008025001042063
:106C4B0004689204B543005034C0E07F203005192E
:106C5B007F30A20472087207500F126C88C204C2F4
:106C6B0008C207C20A7F30800F300703E9C0E01269
:106C7B0069D7300703D0E0F9D0E0B543CC30071724
:106C8B007F30B9100C1269D77F583006077F788098
:106C9B0003B908031269D73004057F2D0269D77F2A
:106CAB0020200AF87F2B2008F322920480CF286E35
:106CBB00756C6C2900D20312699C3003F8C20378FF
:106CCB004330D50108F6026A422D504349581269E8
:106CDB009C2403B405004001E4906CD4931269C862
:0D6CEB00743A1269C8D205754304026B2784
:107136008B2E8A2F8930E4F53AF539F538F537F58F
:1071460035F536E532453345316012EBC0E0EAC02D
:10715600E0E9C0E0AB31AA32A9331270CCAB2E0500
:1071660030E530AA2F7002052F14F9127007F53B8F
:10717600C394094007E53BD3940D40E1E53B642009
:1071860060DBE53BB42D054336038016E53BB42BA7
:1071960005433601800C74FF2530F53074FF352F1A
:1071A600F52FE53460046410703FAB2EAA2FA9308A
:1071B60012700764306009E534702E75340A802930
:1071C600900001127020FF64786004EFB4581343F6
:1071D600360175341074022530F530E4352FF52F5D
:1071E6008007E5347003753408AB2E0530E530AA08
:1071F6002F7002052F14F9127007F53BC3946140F6
:107206000AE53BD3947A5003533BDF74D0253BF514
:107216003BC3940A400CE53B9411406D74F9253B41
:10722600F53BE53BD395345060433601853A3F85BF
:10723600393E85383D85373CAF347E00E4FCFDABF6
:107246003AAA39A938A83712705FC8ECC8C9EDC97F
:10725600CAEECACBEFCBE4FCFDFEEB253BF53AEEDE
:107266003AF539ED39F538EC38F537AF3AAE39AD90
:1072760038FCAB3FAA3EA93DA83CD3126F7550031C
:107286000271EF4336040271EFE53620E003E48035
:107296002DE53245334531601EAB2EE53024FFF92E
:1072A600E52F34FFFAEBC0E0EAC0E0E9C0E0AB311D
:1072B600AA32A9331270CCE53630E20774FFFFFE1E
:1072C600FDFC22E536AF3AAE39AD38AC3730E103D6
:0472D6000270AE2272
:10700700BB010689828A83E0225002E722BBFE0287
:09701700E32289828A83E49322BA
:10702000BB010CE58229F582E5833AF583E0225025
:1070300006E92582F8E622BBFE06E92582F8E2226F
:0D704000E58229F582E5833AF583E4932289
:10704D00BB010689828A83F0225002F722BBFE0122
:02705D00F3221C
:10705F00E88FF0A4CC8BF0A42CFCE98EF0A42CFCD0
:10706F008AF0EDA42CFCEA8EF0A4CDA8F08BF0A44E
:10707F002DCC3825F0FDE98FF0A42CCD35F0FCEBAD
:10708F008EF0A4FEA9F0EB8FF0A4CFC5F02ECD3972
:0F709F00FEE43CFCEAA42DCE35F0FDE43CFC22DF
:0E70AE00C3E49FFFE49EFEE49DFDE49CFC22F3
:1070BC00FAE6FB0808E6F925F0F618E6CA3AF622D5
:1070CC00BB011A89828A83D0F0D0E0F8D0E0F9D0E5
:1070DC00E0FAD0E0FBE8C0E0C0F00271245016E901
:1070EC00F8D083D082D0E0F9D0E0FAD0E0FBC082B7
:1070FC00C08302711BBBFE16E9F8D083D082D0E0AE
:0F710C00F9D0E0FAD0E0FBC082C08302712D22DF
:09711B00EBF608EAF608E9F62299
:09712400EBF0A3EAF0A3E9F0226C
:09712D00EBF208EAF208E9F22293
:00000001FF
